:1000000037010100252CA94873000000828014816B
:10001000988133E6E60009C685050505E389E6FE15
:1000200013351600828052B82A84F52D2A94E52DC6
:10003000E36F85FE52BE46B822E422E00145130577
:10004000C07A01441304407BA2857D2D0145130530
:10005000807BA285552D01451305007CA285226475
:10006000026446BA55A54EB822F44AF052EC5AE85A
:1000700062E46AE0792D630C051A056B130B8B970C
:10008000814B930BC07A014C130C807C856C014D25
:10009000130D807B814D930D007C814A930A007D76
:1000A0000949014A130A107E81499309907E9304FD
:1000B000CB0113044B0101A813B51600238CAC9699
:1000C000892D63060516C145A14626852286B925D8
:1000D000FEAC1D4614813367D6003DC398817D1662
:1000E00085050505E388E6FE1D45A6856A8694819B
:1000F0003367D50025C718827D1505068505E38879
:10010000E6FE1305CB019D456E86148133E7D500CD
:1001100025CB1882FD1505060505E388E6FE1305C7
:10012000CB019D455686148133E7D5002DCF18822B
:10013000FD1505060505E388E6FE03258B009DA851
:100140001D45A28562869881B366E500B5D61C82FE
:100150007D1505068505E308F7FEB9BF1D45A28597
:1001600062869881B366E50099C61C827D150506F6
:100170008505E308F7FE13B51600A38CAC9689B786
:1001800013054B019D4562861881B3E6E50099C6CB
:100190001C82FD1505060505E308F7FE13B51600DC
:1001A000238DAC9631BF03258B0063052501954552
:1001B0006311B5069305CB011D46D2869881B367BE
:1001C000E60081CB9C827D1685068505E308F7FE57
:1001D00039A099456305B5008D456311B5049305B4
:1001E000CB011D46CE869881B367E60081CB9C8209
:1001F0007D1685068505E308F7FED9B59145E3012F
:10020000B5EC9D45E30EB5EA0545A302AB004E856E
:1002100011A80545A38DAC96568529A00545230256
:10022000AB00528581459305807DF92951BD22742B
:100230000279626A426B226C026D4EBE4EB8411169
:1002400022FC4AF852F45AF062EC6AE881499309B8
:10025000C07A014B130B407B814A930A807B814C0F
:10026000930C007C856D938D8D97A9440944054AB4
:10027000014913090078056D130DAD82056C130C4F
:100280001C8405651305C595930575002EC6550597
:100290002AC4FAAD9529FAAE85296685DA85AD219D
:1002A000D93303A58D0063E5A442334525210841D8
:1002B000028501451305107F8121056513054582DF
:1002C000EA859921056513051583EA8535290565B4
:1002D00013057583EA850D2905651305D583EA8520
:1002E0002521056513058587EA85392905651305E7
:1002F0002586E285112901451305007D0564130457
:100300000485A285112101451305107EA285ED2EDD
:1003100001451305907EA285054AFD260565130556
:10032000A5853244A285CD26056513055586A2858F
:10033000E12E0565130505872244A285F126056592
:100340001305D587A2850944A9447D2E05651305AB
:10035000A5885D2623A44D01A5AE03A50D01930537
:10036000F5FF23A8BD006345AA3605651305D58DA5
:1003700061261D4523A4AD00A1AE056503459597F3
:100380006308053405651305D591BD2601451305A0
:10039000107E856593850585852E05651305258663
:1003A000E2859D26056513058587E285B12E0565E5
:1003B00013051583E285892E03A5CD00630D05285D
:1003C00085659385C595B9050565130505872D2EAA
:1003D00085659385259351AC03A50D019305F5FF24
:1003E00023A8BD006346AA2E05651305758C292632
:1003F000154523A4AD00E9AC03A50D019305F5FF58
:1004000023A8BD006346AA2C05651305258DED24A0
:10041000194523A4AD006DAC03C54D0005896304E7
:10042000051823A64D0105651305858EF124254584
:1004300023A4AD00056513057583EA85F1240565E0
:100440001305D583E28579A205650345859705895E
:100450006300052805651305F589792C05651305E5
:100460008587E2855524056513054582E285692C5B
:1004700023A48D00154523A8AD0005651305A585AA
:1004800085659385C595492405651305D58A8565D8
:100490009385458B2DAC03C54D0005896306051476
:1004A00023A60D0005651305858EB924254523A4D3
:1004B000AD00056513054582EA85B9240565130578
:1004C000D583E285B9A203A5CD00630F05140565A8
:1004D0000345B597631C051A03C55D00630A051E35
:1004E00023A60D00A9A205650345A597058963010B
:1004F000051E056513057594012401451305907EBD
:10050000856593850585092423A64D010565130599
:100510002586E285D52A056513057583E285ED22DA
:1005200085659385C595B90505651305D587E92AC0
:10053000056513055595856593852593F122A3825D
:100540000D00114515AA05650345859705896301C9
:10055000051805651305F590452201451305007D35
:100560008565938505854D2223A60D000565130538
:100570008587E285512A056513054582E285692252
:1005800005651305A58585659385C595B52A05651A
:100590001305D58A85659385458BBD22A3810D0002
:1005A00023A48D00E1A805650345B59763020512F4
:1005B00023A64D010565130525903D2A214523A459
:1005C000AD00056513057583EA853D2A05651305AC
:1005D000D583EA85152A056513058587EA852D22C9
:1005E00005651305D587DDA003C55D006302050E13
:1005F00023A60D0005651305558FFD2823A49D0036
:10060000056513054582EA85012205651305D58335
:10061000EA85DD28056513052586EA85F52005654B
:100620001305A585B24565A003C55D0021CD05650F
:100630001305558FD12023A49D000565130515834F
:10064000EA85D92005651305D583EA8575280565F2
:100650001305258695A00565130555868565938543
:10066000C5955D2085659385458B05651305B59218
:10067000612823820D000D4523A4AD00154523A854
:10068000AD00B9A005650345B59739C123A64D0155
:100690000565130525908D20214523A4AD00056532
:1006A00013051583EA858D2005651305D583EA8535
:1006B000A128056513058587EA85B9200565130519
:1006C0005586B2459120056513050587A2452D285D
:1006D00003A58D006D15E36EA4BA05458520A12004
:1006E000930B15008920E36F75FF0145812855B6EE
:1006F000854873000000828091487300000082806A
:10070000AD48730000008280930810087300000059
:10071000828093085008730000008280930870085C
:10072000730000008280732510C08280732500C092
:100730008280930860087300000082800589F3229C
:10074000008093920248B3E2A200739002808280FC
:100750009548730000008280930800087300000031
:100760008280A148730000008280930830087300E3
:10077000000082809308400873000000828000001F
:10078000B202000048040000D8030000F803000093
:100790005A03000096040000C6040000180400007C
:1007A000460500007A030000E604000073656E73DE
:1007B0006F7231004745540073656E736F7232007B
:1007C00073656E736F7233006D657365636F6E0072
:1007D000627574746F6E31006C696768745F6F6EF8
:1007E00000627574746F6E3200627574746F6E336C
:1007F000000A456C657661746F7220436F6E747287
:100800006F6C6C65720A666F72205256436F6E741D
:10081000726F6C6C65720A496E697469616C697A91
:10082000696E6700646F6F723100657874656E641D
:1008300000646F6F723200646F6F72330073656CA7
:1008400000726574726163745F737469636B7900BD
:100850006C696768745F6F6666006C616E74657260
:100860006E317570006C616E7465726E32757000F9
:100870006C616E7465726E32646F776E006C616E5F
:100880007465726E33646F776E000A426F74746FB2
:100890006D20466C6F6F722044656D616E64000A56
:1008A00042464420436F6D706C65746500636869EF
:1008B0006D65310063656C657661746F725F636846
:1008C000696D655F7570000A49646C65206174200C
:1008D00031000A49646C652061742032000A496461
:1008E0006C652061742033000A4D6F76696E672055
:1008F000746F2032000A4D6F76696E6720746F2026
:1009000033000A4D6F76696E6720746F2031000ADC
:10091000417272697665642061742031000A417207
:1009200072697665642061742032006368696D6560
:10093000320063656C657661746F725F6368696DC0
:10094000655F646F776E000A417272697665642034
:0C09500061742033006368696D6533003A
:10095C0035356666353500303033333030006666F9
:10096C003535353500333330303030000000000081
:10097C00000000000000000000000000000000006B
:10098C00000000000000000000000000000000005B
:08099C00000000000000000053
:00000001FF
